:0300000002000EED
:0300030002019F58
:20000B00020196758112D2AFD2A91201A280FE12001B80FBC82581C822C92581C97A002231
:20002B00D083D082CF2581F581CFC082C08322CF2581F581CF22FBE493CB22FCE493FB7492
:20004B000193CC22FAE493F9740193CA2229F9E5F03AFA227C00CB30E7011CCB2275F0009B
:20006B0030E70215F022FDE493FF7401934F7004A3A3800C740293B50510740393B5F00A99
:20008B00E493C0E0740193C0E022A3A3A3A380D7FEEBA4FD8EF0ECA4FCEB8EF0A4C5F02C0F
:2000AB002DC5F02211B58EF0ED22C002C001AAF0F97E007D007F11C3E933F9EA33FADF0867
:2000CB00F5F0E9D001D00222ED33FDEE33FEC3ED9BF5F0EE9C40E0ADF0FED380DBBB0001E7
:2000EB0022C333C5F033C5F0DBF722BB000122C3C5F013C5F013DBF722240280022401C595
:20010B00F03400C5F022C394028003C39401C5F09400C5F0223116F4C5F0F4C5F02245F095
:20012B007022042231784024801A3178401E7014801A3178400E7014800A3178500E8004A0
:20014B00318C6008E4F5F022318C60F8E4F5F00422318C40F780ED318C40F170E780ED313C
:20016B008C40E170E780DD318C50E180D7C39BC5F09C20E70720D207C345F02220D2F9D340
:20018B0022C5F0C39C7003E5F09B22758CDC758A000508320508327400F5087412F50E7451
:2001AB0000F50D7400F50B7400F5097400F50A7400F50F7400F512D2AFD2A8D288740175A7
:2001CB00F00045F070030201FEE5081200687B0112005F12012F45F070030201EB0201D478
:2001EB007400F5081201FF1202A31203851204080201C822E50904F50914E50975F0007B43
:20020B00197C0012017245F070030202A27400F509E50F4408F50FE50A04F50A14E50A754B
:20022B00F0007B027C0012017245F070030202A27400F50AE50F4401F50FE50B04F50B143F
:20024B00E50B75F0007B3C7C0012017245F070030202A27400F50BE50F4402F50FE50D0490
:20026B00F50D14E50D75F0007B3C7C0012017245F070030202A27400F50DE50E04F50E147C
:20028B00E50E75F0007B187C0012017245F070030202A27400F50E22E50F541075F0007B48
:2002AB00007C0012015345F070030202BB1202BC22E50F540175F0007B007C0012015345A8
:2002CB00F0700302031E12031FE50E75F0007B137C0012014B45F0600CE50D75F0007B0026
:2002EB007C0012014B45F070030202F9C297E50E75F0007B167C0012014B45F0600CE50DC5
:20030B0075F0007B007C0012014B45F0700302031ED29722E50F542075F0007B007C0012EC
:20032B00014B45F07003020384E50E75F0007B127C0012014B45F0600CE50D75F0007B0003
:20034B007C0012014B45F07003020359C297E50E75F0007B127C0012014B45F0600CE50D07
:20036B0075F0007B017C0012014B45F07003020384D297E50F4420F50F2212038C1203D118
:20038B0022E50F540875F0007B007C0012015345F070030203D0E50F54F7F50FE50C04F574
:2003AB000C14E50C75F000AB127C0012016A45F070030203D07400F50CE50F4440F50FC2D6
:2003CB00B77402F51122E50F544075F0007B007C0012015345F07003020407E51114F511AE
:2003EB0004E51175F0007B007C0012014B45F07003020407D2B7E50F54BFF50F22E5B054EA
:20040B00011200687B0012005F12014B45F0700302043E7412F50E7400F50D7400F50B7439
:14042B0000F50AE50F4410F50FE50F54DFF50F740AF51222A0
:00000001FF
